:020000040000FA
:02000000D32FFC
:08000800F000030EF100831269
:100010000313F31D48287808FB0B1628FF3E8100C8
:100020007908242086007A08FB001A2881007908C4
:1000300024208600790A1F39F900FC0A0B11710E81
:100040008300F00E700E090082074B3449344334AC
:1000500041340B3409340334033403340334093496
:100060000B344134433449344B34833489348B3436
:10007000C134C334C934CB34CB34CB34CB34C9349E
:10008000C334C1348B34893483348207013402345D
:10009000831203130B184D281F28060800000B10AD
:1000A0002D300102031C5728731381011F28731779
:1000B00081011F28F31E6328F312E530F800013098
:1000C000FB00FA006928F316C830F8000130FB0085
:1000D000FA00080083160313C03081008312031353
:1000E0009630AC0006080B10143026220B1C7B281F
:1000F0006400AC0B72280614F9015A2000308A0003
:10010000F3150B118B160800F601F701F301F4014A
:10011000F5010630EE006B270030722401307224A6
:10012000FF306D06031D0800EC01ED01C626080036
:10013000EC199B28F3286C1FF3286D1CF328741D01
:10014000DC28EE036E08031DA8280630EE00DC282C
:10015000181218166D112030AC23F523F419EE286F
:100160002308243A0319B528AD282430C72199243F
:10017000F419EE285C27AC00ED1EC028A530C72876
:100180006D1FC428A230C728ED1FF32892302C061B
:100190000319CD284630C721AD280330AC23FA20FF
:1001A00024305021F410B201BB24230850210D301B
:1001B0002306031DD428F128ED1CF32808308A00FB
:1001C000CC2000308A00FA20B201EC21AC00003AC9
:1001D0000319F1282C085021B20AE5282130AC235C
:1001E000F32843219221A40A603024060319A401B4
:1001F00076100800ED1DFE28D22100296A20352145
:1002000045308400F3131D21F3133E308400453044
:100210006806031916291D214C308400680603194D
:1002200016291D210730840704080E29F3171D2104
:1002300003305021F030502108000730BB00000887
:10024000AC0001303B06031D2E290310AC0DF31B3F
:100250002C142C0850210630840208000310AC0D29
:100260002C085021840ABB031F29FF30B500B600BB
:1002700081308316031392008312031391018C10B3
:100280006B0870210800FF303506AC00FF303606E1
:1002900050212C085021023070218C1C4D2908005F
:1002A000B3006400ED1969290830B000330C7E21D9
:1002B000B30C031C65297312AF0A8B212F08053A72
:1002C00003196529B00B56290800AF0173168B215D
:1002D000622908308A003308002001308A000800B3
:1002E000AA000630B00073168B2173128B21B00B5D
:1002F000752973168B21AA0B712908000130031888
:10030000B6060310B50CB60C031C08000830B60680
:100310008430B506080064008C1C8B298C10731A7D
:100320005A2008008B12000006100800731B9C293D
:100330003D1CA029BD0AAC293D18A029BD0AAC2945
:100340008C1C9629813083160313920083120313A9
:1003500091018C1003140800C2308316031392001D
:100360008312031391018C1003100800EC18C629A6
:10037000BC001F3C031CC6293C080D3A0319C629C2
:100380003C080A3A0319C629030108003C08741AFC
:10039000CE290C1EC929990064000800B700D62197
:1003A000B20A0800FD010E30AC2308003208FF3C01
:1003B000031C0800AD0AE0293208FF3C031C0800BA
:1003C000F7217319E62937088000080037088317DA
:1003D0008000831373110800AD03F7217319F2290C
:1003E00000080800831700088313731108007311B5
:1003F0003208003C0318052A32083F3C0318092A3A
:1004000032089F3C03180E2A142A32086F3E8400DB
:10041000080001303202A03E840008004030320261
:10042000103E840073150800A0303202903E840014
:1004300073150800FA30A9000000A90B1C2A080057
:10044000AA00C8302622AA0B212A0800A8001A22D6
:100450001A221A221A221A22A80B272A0800D621A9
:10046000B20A0830B000B70C7E21B00B332A080066
:100470000630B100EC21AC000310AC0C2C08203A83
:100480000319442A2C08B621B20AB10B3A2AEC21EE
:10049000B900B90C0F30B90503195A2A2D30C721FC
:1004A0000A303902031C572AB9003130C7213908F4
:1004B000303EC72129083206031D602A2A30C72191
:1004C0000800F3118B12831603138430810083120A
:1004D00003130B108B1528308400E3237310FF30B7
:1004E000B500B6009101C23091008C10BD270318F1
:1004F000C32A9621B40C34087E3A031D762AB4012F
:100500000830B0009621031C8E2AAF0AB40C2F08C5
:10051000053A0319902AB00B822AA42AAF01862A31
:1005200096210318952AAF018B2A962103186B2A6E
:100530003008033A031D6B2AAF01731C7F2A2E0873
:100540000F3C03186B2AB42A731C7314AE0A2E08CE
:10055000FF3A03196B2A2E08023C031C2F2238088D
:10056000B7003408B8007F2AFF30B606B506370852
:100570003606031D6B2A38083506031D6B2A023028
:10058000AE027717F7168B11080077136C1ADB2A67
:100590006C1D08006C1F0800B2013E3084009223DD
:1005A000031CD32ADB2AEC1F0800B201613084004F
:1005B0009223031C08006D1A282BFF30A9000D3070
:1005C000B200ED21B9003918E82A0730B207E12A54
:1005D0003208A8000D3032060319F72AB91BF52A94
:1005E0000730B202ED21B900EA2A3208A90007302B
:1005F000B20038223E30C721B201382228080D3A15
:10060000031D052B0D30B200122B2C30C7210E30EC
:10061000B2003822280832060319122B2C30C721C9
:10062000B20A092B2030C7213C30C7215530C721E1
:100630004930C7213E30C7213A30C7210230B207C6
:10064000AD022D080319372BB20AEC21B621212B5C
:10065000B201D2212D080319372BEC21AC00B20ACC
:1006600008308A002C08002003308A002A2B0E3024
:10067000AC230800F712EC1E08006C1F08002D08C0
:10068000BA000D30B200ED21B9003918902B1430AA
:10069000B200ED21B900B91F552B391808000730F9
:1006A000B207443C031C0800492B0630B202320852
:1006B000A8003E3084009223031C5F2B802BEC1F8C
:1006C00008002808B200613084009223031C08004F
:1006D0002808B2000730BB003E3084000008B70095
:1006E0000310B70D0408A900ED210139B704DC217E
:1006F00029088400BB0B7D2B802BB20A840A6E2B49
:100700002808063EB200ED218038B700DC216A20BF
:100710003521B201ED215021B20ABA0B8A2B4321B7
:10072000922108000730BB000008AA000408AB00B3
:100730000310AA0DED21B400341034082A06031D5D
:10074000AA2B2B088400BB0BA72B03140800B20AAA
:10075000840A942B03100800A800831203170B309F
:100760008F00E7308D0083120313280826271327F4
:10077000831203178D000E088F0083120313CB23FF
:100780000800831203170A308F00A0308D008312F7
:100790000313CB23080013270310FE0DFF1B7E1449
:1007A000FF1303017E06031DDA2B03017F060319E5
:1007B0000800DC2B7E08C72103017F06031DC7212B
:1007C00001302627CB2B80013D3004060319080099
:1007D000840AE32BB2018130B700FF30AB00D62191
:1007E000AB0BF32B0800B20AEF2BAC01F411640041
:1007F0008C1A0C2C0C18FD2BF72B67308F002E3029
:100800008E000C10AC0A70302C06031DF72BF4156B
:100810000800A3018C1E08001A08A30098181B2CBE
:1008200018191E2C0D30230603191A2C6D1D1A2CB5
:100830002308C72108001812181608001A08080013
:10084000613023020318252C08007B302302031C8F
:100850002A2C08002030A3020800AA01BB240D3076
:1008600023060319412C20302306031D412C582C4C
:10087000BB240D30230603195B2C203023060319FB
:100880005B2C30302302031C582C3A30230203180F
:10089000582C3030A3020930AB002A08AA070318ED
:1008A000582CAB0B4E2C2308AA070318582C382CB5
:1008B0000301031408002A08031008000A30262246
:1008C0008C1E642C1A085E2C9818692C18196C2C34
:1008D00008001812181608001A08080023308400AF
:1008E000E3230800AC00693084002C08840700086A
:1008F000A800253084002C08840728088000080000
:10090000771200308A00AB0125302B0784000008E5
:100910000319932C80030008031D932C2B084520FA
:10092000F6042B087224AB0A02302B06031D842C1C
:100930000800B201F523F419B82C2308083A03196A
:10094000A22CA82C0301320603199A2CB2039A2C6C
:100950002308B700D621B20A0A3023060319B82C9F
:10096000033023060319B82C7C303206031D9A2C61
:10097000B701D6210800EC21A300B20AF418202404
:1009800008000408A9000630AB000008AC002030C5
:100990002C060319CD2C2C08C721AB030319D22C2C
:1009A000840AC52C2D30C721840A0F300005AC0005
:1009B0000A302C02031CE02C3130C7210A30AC0273
:1009C00030302C07C7212908840008008312031740
:1009D0000D308F0079308D0083120313B201BB24D8
:1009E0001327AC0023060319082D2C082302031C2F
:1009F000062D013026271327AC0000302C060319E2
:100A0000062D01302E272C082627F02C0310080075
:100A1000023026271327AC00FF302C06031DEF2CD5
:100A2000013026271327031408008C1E0800F41435
:100A30009924E62403181E2D0230BD2EAC0005308B
:100A40008A002C0882076D2D8D2DA02D5E2DD42DB2
:100A5000D22DD62DD92DDF2DEA2DF92DDC2DFB2D14
:100A6000E62D6B2DF72DC72D432D8B2DAA2EAD2EE8
:100A7000AF2EA42EA72E452DB12EB52EB92E5A2D50
:100A8000472DCE2DD02D6C14BF2E6C10BF2E2D24D3
:100A90000318BD2EAC000D302306031DBD2EC9303A
:100AA0002C020318BD2E00302C060319BD2E2C0875
:100AB000EB00BF2E1D30AC23AC27BF2E613084006D
:100AC000CD260301040603196B2D0D302306031DEB
:100AD0006B2DEC17BF2EEC13BD2E2D240318BD2E4D
:100AE000AC000D302306031DBD2E3D302C02031833
:100AF000BD2E00302C060319882D0F302C02031C4C
:100B00000310AC0D2C0DE90003017224EC15BF2E6F
:100B1000EC11E901BF2EC123BF2E0E30AC236C1F98
:100B20009A2D6D1C9D2D5E24F7147710F41004305F
:100B3000AC2308000B30AC23BD2E0A30AC23BD2EF5
:100B40004530A90029088400CD26030104060319B5
:100B5000C72D5A302906031DB22D0D302306031967
:100B6000CA2DC72D0D3023060319CA2D20302306A8
:100B7000031DC72DBB2456302306031DC72DBB24E0
:100B800020302306031DC72D0730A907A22D6D10A5
:100B9000E801BD2E6D142908E800BF2EEC10BF2E11
:100BA000EC14BF2EEC16BF2EEC12BF2E6C166C117F
:100BB000BF2E6C156C12BF2E6C126C11BF2E3E3006
:100BC0008400CD2603010406031DE82D6C13BD2E01
:100BD0006C17BF2E6430AB00F410BB2423089127A0
:100BE000AB0A2308003A031DED2DED14BF2EED10C6
:100BF000BF2E8327BF2EEC1C002E2530AC23022EE7
:100C00002430AC236D19072E1230AC23092E11307D
:100C1000AC236C180E2E2230AC23102E2330AC23C4
:100C20001E30AC2308308A006B08822003308A0013
:100C30000E30AC231630AC23ED1E212E1730AC2322
:100C4000292E6D1F262E1B30AC23292EED171C30AC
:100C5000AC230E30AC23ED19352E6D1A322E133025
:100C6000AC23382E1430AC23382E1530AC23382E5C
:100C70000E30AC230630AC236C1A422E6C19442E75
:100C80001930452E0730452E1830AC23EC1A4B2E68
:100C90000930AC234D2E0830AC23EC1D5D2E1030F6
:100CA000AC236908AC0008308A000310AC0C2C0C93
:100CB000822003308A000E305E2E0F30AC230A30C3
:100CC000AC236D18662E0E30AC23782E4530840090
:100CD000C1240730840704086802031C762E2030E4
:100CE000C7215630C7212030C721682E0E30AC23D3
:100CF0000B30AC236C1F7F2E3E308400C1240E309D
:100D0000AC230C30AC23EC1F882E61308400C1244E
:100D10000E30AC230D30AC23ED1CA12E6430AB00A3
:100D20002B08831203178D00831603170C148312EC
:100D300003170C08831203130319BF2EC721AB0A34
:100D4000902E0E30AC23C12E6D16ED11BF2EED1579
:100D50006D12BF2EED116D12BF2E6D15BF2E6D11D0
:100D6000BF2EED166D13ED13BF2E6D17ED12ED13A3
:100D7000BF2EED176D13ED12BF2E0530C02E0330C0
:100D8000AC230130AC235E24F41008006C16EC1682
:100D90006D15ED164030EB0008000408A800073080
:100DA000B10020308000840AB10BD12E28088400C5
:100DB000B101BB242D3023060319F72E0D30230675
:100DC0000319F12E203023060319F12E28083107CC
:100DD000840023088000B10A3108073A031DD92E88
:100DE000112F063028078400303080000E2F2D246C
:100DF0000318112F303EAC0040302C020318112F85
:100E00000630280784002C0880000D3023060319C3
:100E10000E2F2030230603190E2F112F28088400CF
:100E2000080084010800831603178C170C140000B7
:100E30000000831203170C08FF000E08FE000C08C8
:100E4000831603178C1383120313080083120317EE
:100E50008D0703188F0A83120313080083120317E8
:100E60008D02031C8F038312031308008C1E0800DD
:100E70009924F419552F033023060319552F0D30EB
:100E8000C7210A30C721B201FA20F410BB24033075
:100E900023060319552F030123060319522F230894
:100EA0005021462F4321922108009221F7107714F8
:100EB0005E240130AC230800B201BB01EC21A30089
:100EC000202406303206031D672F3B080800B20AB3
:100ED0002308BB075E2FAB013E3084002B08831232
:100EE00003178D00831603178C010C14831203174C
:100EF0000C088312031380002F302B0603190800FF
:100F0000840AAB0A6E2FAB013E30840083120313B8
:100F1000000891272F302B0603190800840AAB0A1A
:100F2000862F0D12831203178C00831203132B08D4
:100F3000831203178D00831603170C158B1355307E
:100F40008D00AA308D008C140C11831203130D1E1A
:100F5000A72F0D128B1708006A2035216400092481
:100F6000203023060319B92F033023060319BB2FA2
:100F7000AE2F5A20AE2F9221080064000C18C12F0A
:100F8000CF2F67308F002E308E000C10A70AEF3065
:100F90002706031DCF2F7716A7010314080003109F
:100FA0008C1A031408006E24EA23842008308A0077
:100FB0005F2007308A00F717851EE42F0030AC232E
:100FC0000130AC237714E92F74156C126C111F30AB
:100FD000AC23640077181525F7183627771A802474
:100FE00076189820F71B6122F71A3A23771BC5223F
:020FF000E92FE7
:10100000132001308A002030C72108308A00FD0AF1
:101010000F307D05031D080003308A000E30AC231D
:1010200008308A000800AA00AB00F030AB050310BE
:10103000AB0CAB0CAB0CAB0C2B083020AB00013075
:101040008A002B08C72108308A000F302A0530207B
:10105000AB0001308A002B08C72108308A00080045
:101060008207303431343234333434343534363426
:1010700037343834393441344234433444344534D9
:1010800046340630831603139C001F309B00F73054
:101090008500343086008312031385018601080021
:1010A0000730831603139C0000309B00FF3085003F
:1010B000FD3086008312031385018601080050204D
:1010C00041208316031318152030990098168312B7
:1010D000031398171816313090000F3092000B1739
:1010E0008B17031A7B2803308A000E30AC231A308A
:1010F000AC2308308A00831203171730850083124F
:1011000003130800AC00AB01F412A901AC1F912835
:1011100001308A002D30C72108308A00AB0AAC09A3
:10112000AC0A08308A0004302B060319BA280330B1
:101130002B060319A3282B08C7202C02031CA62862
:10114000AC00A90A9128F41ABA28AF28030129068D
:101150000319AB28AF28F518AF28F41EB7280130C3
:101160008A00F41630302907C72108308A00A90107
:10117000AB0A9128751CC52801308A002E30C72182
:101180003530C72108308A007510F5100800820735
:1011900064340A3401340034502074138518472114
:1011A00041206430AA002A08831203178D00831699
:1011B00003170C14831203170C0883120313B700D0
:1011C0005C3A031D2C29AA0A831203178D0A831681
:1011D00003170C14831203170C0883120313B700B0
:1011E000733A031DF82874162408822074123529D6
:1011F000741F35293708683A031D0629741621081B
:1012000037216C1C422282207412352937086C3A2F
:10121000031D12297416220837216C1C42228220D9
:10122000741235293708743A031D1E2974162008D4
:1012300037216C1C42228220741235293708613A0A
:10124000031D2B2974162008372142227510F5142E
:10125000822074123529000001308A00D62109301D
:101260008A00370803190800B20AAA0AD3287510A1
:10127000AC002C187514AC1B402903102C0C080072
:10128000AC09AC0A0310AC0CAC092C0A0800A8018C
:10129000A901BF21741F9329CC3016224430162295
:1012A000861402308A000430202209308A00861019
:1012B000BF21CC301622BE3016220930B100BD014C
:1012C000EA21340809303106031D69293408A000D9
:1012D000762908303106031D76293408AC00031046
:1012E000AC0CA00CAC0CA00CAC0CA00CA821B10B4D
:1012F000602903013D0603197F297413080000309B
:101300002406031D87292008A200A1009329220892
:10131000942103188D292008A20021089421031C80
:1013200093292008A1000800A800A01B9E29A81B43
:10133000A629280820020318A629A429A81FA42941
:10134000280820020318A629031008000314080027
:101350000830AB003408A80028080139A900B421DE
:10136000A80CAB0BAC29080029083D060139BC00CC
:101370000310BD0C3C1CBE298C30BD060800831632
:1013800085148312A90174138312851083168510A6
:101390008312FE308F0095308E000A308A009C2226
:1013A00009308A00831685148312FF308F00CE30F7
:1013B0008E000A308A009C2209308A00851C74172E
:1013C000FE308F00DE308E000A308A009C22093009
:1013D0008A0000340830AA00831285108316851015
:1013E0008312FF308F00FD308E000A308A009C226D
:1013F00009308A00831685148312FF308F00FE3077
:101400008E000A308A009C220A308A0005080239C0
:10141000FF3EB40CFF308F00DD308E000A308A00B2
:101420009C220A308A00AA0BEC290034B400083050
:10143000AA0083128510831685108312FF308F0057
:10144000FD308E000A308A009C220A308A00B40CDB
:1014500003188514FF308F00D5308E000A308A00C3
:101460009C220A308A00831685148312FF308F0075
:10147000FF308E000A308A009C220A308A00AA0BB4
:10148000192A0034A800A900831203170A308F001C
:1014900069308D0083120313A81F522A2808A9005F
:1014A000A909A90A07308A00290826271327A900B5
:1014B0000A308A007518A90A7510291875140310C6
:1014C000A90CA81B662A2030290708002908203CFF
:1014D00008000000030007000A000E0012001500BB
:1014E00019001C002000240027002B002E003200D1
:1014F000360039003D004000440048004B004F00DA
:10150000520056005A005D006100640068006C00E3
:101510006F00730076007A007E00810085008800ED
:101520008C009000930097009A009E00A200A500F6
:10153000A900AC00B000B4000C100C1C9D2A0800DF
:101540000D000A00EF21ED36EE3073322810E93B32
:10155000683A6510613CF0366536BA1400100D002B
:101560000A00CF2156272D104310EE37653B733903
:10157000A032EF3665320D000A004521C320CE2788
:1015800028106531E330EE376510653B79396E1010
:10159000AD146E10B01E6910A039E6372033EE305E
:1015A0002032BC183C37301B6D10EE3480390D00F2
:1015B0000A005421D822202A6214653A743C421051
:1015C000E237AD14B0182018E831F230A039E13616
:1015D000003C0D000A00C12149265221D420A0223E
:1015E0004314EC30E2346139653A4D10E437A032EF
:1015F000A016652AF439EE34A033EE27793680142C
:101600000D000A004922C9236538F43028106932D8
:10161000E9336F102F37E63729330D000A004922CE
:10162000D0292D104410F3346C38F93061106C3629
:101630006310ED37E136643780390D000A00C322AC
:101640004F242810E3326F346F102F37E6372933D9
:101650000D000A0049235426D2222810EE37EF1736
:101660006633AD146610EC34653A2039F03A6939C6
:101670007437E23065367410F232E936613720365D
:10168000E831F23080390D000A00D023A029671418
:1016900073382410D023C723AF20471247284C2685
:1016A000A417D0234D29A9210D000A00CF266927B0
:1016B0006F3A20396D14EE3761106C36ED17AF328A
:1016C000E63729330D000A00D926CC20C124A029F1
:1016D0006D14E13C6936F3307710E434B132B11661
:1016E00080140D000A00D926C1214C262810F93695
:1016F000E1316C366C10343D7937B81680140D002A
:101700000A0045284D29281045284D2980140D0030
:101710000A00452AD026F232F430F23AA03274148C
:10172000ED3220382F33A9310D000A00522AE33060
:10173000A032741420396D3CF434F217F631A01441
:10174000A0166F23203965327531E733EE34A033AC
:10175000EE3779360D000A00582A45224126A02C82
:101760007414643CEC32F9306E1030106E1E321E70
:1017700031186E107310F432A03965326136A03C16
:101780006C33E73080390D000A00CE2A5228D42766
:10179000A027751470376F396F3A67107338B331FB
:1017A0002018203BE93B6532AD18A018203BE93BEF
:1017B00065322D1929192D1033106410E734F334D4
:1017C0006D10F8300D000A000D000A0000000D0C2D
:1017D000400C460C480C4C0C620C660C6B0C700CEC
:1017E0007A0C840C890C8E0C930C970C9A0CA20C1E
:1017F000AB0CB20CB90CBF0CC50CCC0CCF0CD30C81
:10180000D70CDC0CEB0CEF0CF30C0C0D110D280DB0
:10181000380D510D5B0D650D6F0D0D000A00C22BCB
:10182000571CC1234D10C427CD224526D32954105F
:10183000432756103210321700180D000A005A269E
:101840004E1AA02C323B33172018B819301A201822
:101850007031A0396F3320396F247536203CB126A2
:10186000301800180D000A00792A65384810CC227B
:1018700020286F332039EE246F330D000A0000005A
:101880000D000A00ED313A32001000003F00000068
:101890000D000A00CB2700000D000A002A152015B4
:1018A0004310EE37653B7339A032EF2665322016C0
:1018B000F4312036A0216F3A4510693C003A0D0002
:1018C0000A0000000D000A00801F0000CF266927D3
:1018D0006F3A20390000CC2000260D000A000000DD
:1018E0004922C9236538F430F2324F1000270D0029
:1018F0000A0000004922C9236538F430F2324F1043
:1019000046230D000A000000CE2A5228D427A02723
:101910000000D926C1214C2600100000D926CC2079
:10192000C124A02900005421D822202A00000D0043
:101930000A0000004521C320CE274F1066330D005A
:101940000A0000004521C320CE274F102037D622A1
:10195000D222A02C0000C3224F244F1000270D00DC
:101960000A000000C3224F244F1046230D000A0036
:101970000000522AE330A032C62700230000522A7A
:10198000E330A0324329002B0000522AE330A0327A
:101990005810C926002A0000D023A02900004712B1
:1019A0005228C3260000C5260D000A000000C627E5
:1019B00000230D000A000000E12B633A20346F225F
:1019C000A033692AE53620396123EC34F23A8032BB
:1019D0000D000A000000471247284C26000047125D
:1019E0004728C1230000E12169367231F430A0326A
:1019F000EF2665322017D0297410A0376F3AE733ED
:101A00006536A01DF4312036A0216F3A4510693C9F
:101A1000003A0D000A000000582A45224126A02C59
:101A200000000D000A00D023A029EF2665325716CA
:101A3000E930693A67376610F2374210E132EF3128
:101A40002037692AE5362E3900170D000A000000FC
:101A50000D000A00E529F230E831EE34A0336F338F
:101A60002039D023A029F527703AF43A201D000030
:101A70000D000A00492AC526D527212A2E17E12B59
:101A8000F434EE34A0336F3320396527743C4210B0
:101A9000E132EF312037692AE53600390D000A00BE
:101AA0000000452AD026F232F430F23AA032002368
:101AB0000D000A000000452AD026F232F430F23A36
:101AC000A03280210D000A0000000D000A006923E9
:101AD0007436F2324F1000270D000A0000000D008E
:101AE0000A0069237436F2324F1046230D000A00B3
:101AF000000042342C3445341A3441340034433429
:101B000000344F3400344E34003420340034453433
:101B100000345634003445340034523400345934DF
:101B2000003420340034FF3400345434003445345D
:101B3000003458340034543400340D340434FF3449
:101B40000F3420340034FF34093443341E3441341C
:101B500012344C34003449340034423400345234AA
:101B60000034413400345434003445340034FF34FC
:101B70001C344F3400344E340034563400340D34A9
:101B80000034FF34013444342234493400344734BF
:101B9000163449340034203400344F340034463491
:101BA0000834463400340D340034FF3404344E34E9
:101BB00000340D340034FF340534533400345034D1
:101BC00000340D340034FF340C3445341A344334BB
:101BD0000034483400344F340034203400344F345F
:101BE000003446340834463400340D340034FF34B5
:101BF00015344E3400340D340034FF34143446347C
:101C00001E34493400344C340034543400344534E8
:101C1000003452340034203400344F34003446341D
:101C20000834463400340D340034FF341F344E344D
:101C300000340D340034FF341E344734243450341F
:101C40000034533400342034003424340034473416
:101C500000345034003447340E34473406344134B1
:101C60000034FF341B344C3400344C340034FF3423
:101C70001A34523400344D34003443340034FF34C9
:101C8000193448340C34453400344C340034503466
:101C900000340D340034FF3412344D3444344F34A6
:101CA0001E344E34003420340034413408344C3473
:101CB00000344C340034FF3406344D34063445349B
:101CC0000034FF3407344F34003446340034463493
:101CD00000340D340034FF340B34593400344134B3
:101CE00012344C3400344934003441340034533419
:101CF00000340D340434FF340E3420340034FF3407
:101D0000033443340034413400344C3400344C3414
:101D100000340D340434FF340D3420340034FF34E7
:101D2000083450340C3445340034523400344D34CB
:101D300000340D340034FF340A3454344A3445340A
:101D400014344D34003450340034203400344334DF
:101D500006340D340034FF341134463400340D346D
:101D60000034FF34183452342434203400344F34D7
:101D70000A3446340034463400340D340034FF3421
:101D8000133452340A3443340034563400340D349E
:101D90000034FF341634583400344D3400344934A0
:101DA0000034543400340D340034FF3417345834C4
:101DB000003444340034453400344C34003441346D
:101DC00000345934003420340034FF341D34553489
:101DD00000344E34003450340034523400344F3424
:101DE0000034543400344F3400340D340434FF34A0
:0A1DF000103420340034FF340234B4
:02400E000A3F67
:02401000FC3F73
:00000001FF
